
 TOOLHELP

 Start     Length     Name                   Class
 0001:0000 02DC0H     _TEXT                  CODE
 0002:0000 00010H     NULL                   BEGDATA
 0002:0010 000C4H     _DATA                  DATA
 0002:00D4 00000H     CDATA                  DATA
 0002:00D4 00000H     XIFB                   DATA
 0002:00D4 00000H     XIF                    DATA
 0002:00D4 00000H     XIFE                   DATA
 0002:00D4 00000H     XIB                    DATA
 0002:00D4 00000H     XI                     DATA
 0002:00D4 00000H     XIE                    DATA
 0002:00D4 00000H     XPB                    DATA
 0002:00D4 00000H     XP                     DATA
 0002:00D4 00000H     XPE                    DATA
 0002:00D4 00000H     XCB                    DATA
 0002:00D4 00000H     XC                     DATA
 0002:00D4 00000H     XCE                    DATA
 0002:00D4 00000H     XCFB                   DATA
 0002:00D4 00000H     XCF                    DATA
 0002:00D4 00000H     XCFE                   DATA
 0002:00D4 0000CH     DBDATA                 DATA
 0002:00E0 00000H     CONST                  CONST
 0002:00E0 00019H     HDR                    MSG
 0002:00F9 00082H     MSG                    MSG
 0002:017B 00002H     PAD                    MSG
 0002:017D 00001H     EPAD                   MSG
 0002:0180 00000H     _BSS                   BSS
 0002:0180 00000H     XOB                    BSS
 0002:0180 00000H     XO                     BSS
 0002:0180 00000H     XOE                    BSS
 0002:0180 00040H     c_common               BSS

 Origin   Group
 0002:0   DGROUP

 Address   Export                  Alias

 0001:2D24 CLASSFIRST              CLASSFIRST
 0001:2D31 CLASSNEXT               CLASSNEXT
 0001:0418 GLOBALENTRYHANDLE       GLOBALENTRYHANDLE
 0001:04AA GLOBALENTRYMODULE       GLOBALENTRYMODULE
 0001:0318 GLOBALFIRST             GLOBALFIRST
 0001:0582 GLOBALHANDLETOSEL       GLOBALHANDLETOSEL
 0001:02A2 GLOBALINFO              GLOBALINFO
 0001:039A GLOBALNEXT              GLOBALNEXT
 0001:201A INTERRUPTREGISTER       INTERRUPTREGISTER
 0001:20CA INTERRUPTUNREGISTER     INTERRUPTUNREGISTER
 0001:0964 LOCALFIRST              LOCALFIRST
 0001:0914 LOCALINFO               LOCALINFO
 0001:09F0 LOCALNEXT               LOCALNEXT
 0001:13B2 MEMMANINFO              MEMMANINFO
 0001:288C MEMORYREAD              MEMORYREAD
 0001:2A34 MEMORYWRITE             MEMORYWRITE
 0001:0B96 MODULEFINDHANDLE        MODULEFINDHANDLE
 0001:0B1E MODULEFINDNAME          MODULEFINDNAME
 0001:0A98 MODULEFIRST             MODULEFIRST
 0001:0AE2 MODULENEXT              MODULENEXT
 0001:1B30 NOTIFYREGISTER          NOTIFYREGISTER
 0001:1BE6 NOTIFYUNREGISTER        NOTIFYUNREGISTER
 0001:0FA6 STACKTRACECSIPFIRST     STACKTRACECSIPFIRST
 0001:0F5A STACKTRACEFIRST         STACKTRACEFIRST
 0001:100A STACKTRACENEXT          STACKTRACENEXT
 0001:1210 SYSTEMHEAPINFO          SYSTEMHEAPINFO
 0001:0D42 TASKFINDHANDLE          TASKFINDHANDLE
 0001:0CBC TASKFIRST               TASKFIRST
 0001:0DCC TASKGETCSIP             TASKGETCSIP
 0001:0D00 TASKNEXT                TASKNEXT
 0001:0D9A TASKSETCSIP             TASKSETCSIP
 0001:0DF8 TASKSWITCH              TASKSWITCH
 0001:26C8 TERMINATEAPP            TERMINATEAPP
 0001:2C76 TIMERCOUNT              TIMERCOUNT
 0001:018A WEP                     WEP

  Address         Publics by Name

 0000:0000  Imp  ALLOCCSTODSALIAS     (KERNEL.170)
 0001:22BA       CASRQ_HANDLER
 0001:2D24       CLASSFIRST
 0001:2D31       CLASSNEXT
 0001:2349       COMMONINTERRUPTENTRY
 0001:1E5F       DECODENOTIFICATION
 0001:25B3       DIH_30STDCHAINON
 0001:249C       DIH_BADSTACK
 0001:252E       DIH_CALLBACKRESTART
 0001:25D9       DIH_CHAINON
 0001:23EA       DIH_DPMICHAINON
 0001:24F4       DIH_DPMIRESTART
 0001:2639       DIH_EMDPMIRESTART
 0001:25FD       DIH_EMULATEDPMI
 0001:242F       DIH_ENOUGHROOMONSTACK
 0001:2413       DIH_EXCEPTION
 0001:23FF       DIH_FOUND
 0001:255E       DIH_NEXTNOTFOUND
 0001:25F4       DIH_NOCHAINADDR
 0001:23E2       DIH_NOTCASRQ
 0001:23A0       DIH_NOTPVGPFAULT
 0001:25A7       DIH_NUKEAPP
 0001:257E       DIH_NUKEIT
 0001:2669       DIH_REBUILDDPMIFRAME
 0001:2506       DIH_SKIPDPMI
 0001:2463       DIH_STACKOK
 0000:0000  Imp  DIRECTEDYIELD        (KERNEL.150)
 0001:22C4       DIV0_HANDLER
 0002:003A       DWCASRQCSIP
 0000:0000  Imp  FATALAPPEXIT         (KERNEL.137)
 0000:0000  Imp  FREESELECTOR         (KERNEL.176)
 0000:0000  Imp  GETCURRENTTASK       (KERNEL.36)
 0000:0000  Imp  GETFREESYSTEMRESOURCES (USER.284)
 0000:0000  Imp  GETMODULEHANDLE      (KERNEL.47)
 0000:0000  Imp  GETPROCADDRESS       (KERNEL.50)
 0000:0000  Imp  GETTICKCOUNT         (USER.13)
 0000:0000  Imp  GETVERSION           (KERNEL.3)
 0001:0418       GLOBALENTRYHANDLE
 0001:04AA       GLOBALENTRYMODULE
 0001:0318       GLOBALFIRST
 0001:0582       GLOBALHANDLETOSEL
 0001:02A2       GLOBALINFO
 0000:0000  Imp  GLOBALLOCK           (KERNEL.18)
 0000:0000  Imp  GLOBALMASTERHANDLE   (KERNEL.28)
 0001:039A       GLOBALNEXT
 0000:0000  Imp  GLOBALUNWIRE         (KERNEL.112)
 0001:2260       GP_HANDLER
 0001:226A       GP_STDMODEHANDLER
 0001:1741       HELPERGETSEGNUMBER
 0001:14B5       HELPERGLOBALTYPE
 0001:164E       HELPERGRABSELECTOR
 0001:1482       HELPERHANDLETOSEL
 0001:177B       HELPERPDBTOTDB
 0001:1656       HELPERRELEASESELECTOR
 0001:1703       HELPERSEGLEN
 0001:1665       HELPERSETSIGNALPROC
 0001:1683       HELPERSIGNALPROC
 0001:14A6       HELPERVERIFYLOCHEAP
 0001:1468       HELPERVERIFYSEG
 0002:00B0       HGDI
 0001:22A6       INT1_HANDLER
 0001:22B0       INT3_HANDLER
 0001:2260       INTERRUPTHANDLER
 0001:26AE       INTERRUPTINFO
 0001:218A       INTERRUPTINIT
 0001:2166       INTERRUPTISHOOKED
 0001:201A       INTERRUPTREGISTER
 0001:2218       INTERRUPTUNINIT
 0001:20CA       INTERRUPTUNREGISTER
 0002:005C       INTINFO
 0001:01D6       KERNELTYPE
 0001:016A       LIBENTRY
 0000:0000  Imp  LOCALALLOC           (KERNEL.5)
 0001:0964       LOCALFIRST
 0000:0000  Imp  LOCALFREE            (KERNEL.7)
 0001:0914       LOCALINFO
 0000:0000  Imp  LOCALINIT            (KERNEL.4)
 0001:09F0       LOCALNEXT
 0002:00BE       LPCHAINCSIP
 0002:003E       LPFNOLDPROC
 0002:00B6       LPFNPV
 0002:00AC       LPGDIFLAG
 0002:00BA       LPOLDHANDLER
 0000:0000  Imp  LSTRCMP              (USER.430)
 0001:2C30       MAKEALIAS
 0001:13B2       MEMMANINFO
 0001:288C       MEMORYREAD
 0001:2A34       MEMORYWRITE
 0001:0B96       MODULEFINDHANDLE
 0001:0B1E       MODULEFINDNAME
 0001:0A98       MODULEFIRST
 0001:0AE2       MODULENEXT
 0001:1ABF       NEXTLRU286
 0001:08A2       NEXTLRU386
 0001:1D4A       NOTIFYHANDLER
 0001:1CB6       NOTIFYINIT
 0001:1C92       NOTIFYISHOOKED
 0001:1B30       NOTIFYREGISTER
 0001:1E03       NOTIFYRIPHANDLER
 0001:1D0D       NOTIFYUNINIT
 0001:1BE6       NOTIFYUNREGISTER
 0000:0000  Imp  OUTPUTDEBUGSTRING    (KERNEL.115)
 0000:0008  Abs  pAtomTable
 0001:2288       PF_HANDLER
 0001:2292       PF_STDMODEHANDLER
 0000:0006  Abs  pLocalHeap
 0000:0000  Imp  POSTAPPMESSAGE       (USER.116)
 0000:000E  Abs  pStackBot
 0000:000C  Abs  pStackMin
 0000:000A  Abs  pStackTop
 0000:0000  Imp  REGISTERPTRACE       (KERNEL.202)
 0002:0004       rsrvptrs
 0001:084E       SELTOARENA386
 0001:2274       SF_HANDLER
 0001:227E       SF_STDMODEHANDLER
 0001:2782       SIGNALREGISTER
 0001:2816       SIGNALUNREGISTER
 0001:10EE       STACKFRAMEFIRST
 0001:117A       STACKFRAMENEXT
 0001:0FA6       STACKTRACECSIPFIRST
 0001:0F5A       STACKTRACEFIRST
 0001:100A       STACKTRACENEXT
 0002:00D0       STKHQQ
 0001:1210       SYSTEMHEAPINFO
 0001:0D42       TASKFINDHANDLE
 0001:0CBC       TASKFIRST
 0001:0DCC       TASKGETCSIP
 0001:0EA6       TASKINFO
 0001:0D00       TASKNEXT
 0001:0D9A       TASKSETCSIP
 0001:0DF8       TASKSWITCH
 0001:26C8       TERMINATEAPP
 0001:2C76       TIMERCOUNT
 0001:0010       TOOLHELPLIBMAIN
 0001:0E76       TS_FROMYIELD
 0001:229C       UD_HANDLER
 0001:12A2       USERGDIDGROUP
 0001:12CE       USERGDISPACE
 0001:1320       USERGDITYPE
 0001:181B       WALK286
 0001:17A8       WALK286COUNT
 0001:17D3       WALK286FIRST
 0001:18E4       WALK286HANDLE
 0001:19F7       WALK286VERIFYLOCHEAP
 0001:0615       WALK386
 0001:0596       WALK386COUNT
 0001:05C1       WALK386FIRST
 0001:06D5       WALK386HANDLE
 0001:07F2       WALK386VERIFYLOCHEAP
 0001:1955       WALKLOC286
 0001:1907       WALKLOC286COUNT
 0001:192E       WALKLOC286FIRST
 0001:074A       WALKLOC386
 0001:06FC       WALKLOC386COUNT
 0001:0723       WALKLOC386FIRST
 0002:0038       WCASRQFLAG
 0001:018A       WEP
 0000:0000  Imp  WOW16CALL            (KERNEL.500)
 0002:0180       _edata
 0002:01C0       _end
 0002:018C       _hGDIHeap
 0002:0196       _hMaster
 0002:01AE       _hUserHeap
 0002:01A2       _lpfnFatalExitHook
 0002:019A       _lpfnGetFreeSystemResources
 0002:01AA       _lpfnGetUserLocalObjType
 0002:0192       _lpfnNotifyHook
 0002:0186       _lpfntimeGetTime
 0002:0182       _lpfnUserSeeUserDo
 0002:0190       _npdwSelTableStart
 0002:01B4       _NPINTHEAD
 0002:01A8       _NPNOTIFYHEAD
 0002:018A       _NPNOTIFYNEXT
 0002:01A0       _NPSIGNALHEAD
 0002:01BC       _npwExeHead
 0002:01B8       _npwSelTableLen
 0002:0198       _npwTDBCur
 0002:018E       _npwTDBHead
 0002:01BE       _segKernel
 0002:0010       _szKernel
 0002:01A6       _WINTINSTALLED
 0002:0180       _wLibInstalled
 0002:01B2       _wLRUCount
 0002:01B6       _WNOTIFYINSTALLED
 0002:019E       _wSel
 0002:01BA       _WSIGNALINSTALLED
 0000:0000  Imp  _WSPRINTF            (USER.420)
 0002:01B0       _wTHFlags
 0000:9876  Abs  __acrtmsg
 0000:9876  Abs  __ACRTUSED
 0000:9876  Abs  __acrtused2
 0000:D6D6  Abs  __aDBdoswp
 0002:00D2       __adbgmsg
 0002:00D8       __aDBrterr
 0000:0000  Imp  __AHINCR             (KERNEL.114)
 0002:00E8       __caption
 0002:0180       __edata
 0002:01C0       __end
 0000:9876  Abs  __fptaskdata
 0001:2D44       __fstrncpy
 0000:0000  Imp  __MOD_COMMDLG        (KERNEL.532)
 0000:0000  Imp  __MOD_DGDI           (KERNEL.525)
 0000:0000  Imp  __MOD_DKERNEL        (KERNEL.521)
 0000:0000  Imp  __MOD_DUSER          (KERNEL.523)
 0000:0000  Imp  __MOD_GDI            (KERNEL.524)
 0000:0000  Imp  __MOD_KERNEL         (KERNEL.520)
 0000:0000  Imp  __MOD_KEYBOARD       (KERNEL.526)
 0000:0000  Imp  __MOD_MMEDIA         (KERNEL.531)
 0000:0000  Imp  __MOD_SHELL          (KERNEL.528)
 0000:0000  Imp  __MOD_SOUND          (KERNEL.527)
 0000:0000  Imp  __MOD_TOOLHELP       (KERNEL.530)
 0000:0000  Imp  __MOD_USER           (KERNEL.522)
 0000:0000  Imp  __MOD_WINSOCK        (KERNEL.529)
 0001:2D6E       __NMSG_TEXT
 0001:2D99       __NMSG_WRITE
 0001:2D41       __wflags
 0000:0000  Imp  __WINFLAGS           (KERNEL.178)
 0002:00DA       ___aDBexit
 0002:00D6       ___aDBswpchk
 0002:00D4       ___aDBswpflg

  Address         Publics by Value

 0000:0000  Imp  GETCURRENTTASK       (KERNEL.36)
 0000:0000  Imp  ALLOCCSTODSALIAS     (KERNEL.170)
 0000:0000  Imp  GETPROCADDRESS       (KERNEL.50)
 0000:0000  Imp  GLOBALLOCK           (KERNEL.18)
 0000:0000  Imp  GETTICKCOUNT         (USER.13)
 0000:0000  Imp  __MOD_SOUND          (KERNEL.527)
 0000:0000  Imp  __MOD_DKERNEL        (KERNEL.521)
 0000:0000  Imp  OUTPUTDEBUGSTRING    (KERNEL.115)
 0000:0000  Imp  POSTAPPMESSAGE       (USER.116)
 0000:0000  Imp  __MOD_SHELL          (KERNEL.528)
 0000:0000  Imp  GLOBALMASTERHANDLE   (KERNEL.28)
 0000:0000  Imp  __MOD_TOOLHELP       (KERNEL.530)
 0000:0000  Imp  __MOD_MMEDIA         (KERNEL.531)
 0000:0000  Imp  DIRECTEDYIELD        (KERNEL.150)
 0000:0000  Imp  LOCALINIT            (KERNEL.4)
 0000:0000  Imp  FREESELECTOR         (KERNEL.176)
 0000:0000  Imp  __MOD_COMMDLG        (KERNEL.532)
 0000:0000  Imp  __WINFLAGS           (KERNEL.178)
 0000:0000  Imp  LOCALALLOC           (KERNEL.5)
 0000:0000  Imp  FATALAPPEXIT         (KERNEL.137)
 0000:0000  Imp  __MOD_USER           (KERNEL.522)
 0000:0000  Imp  GETFREESYSTEMRESOURCES (USER.284)
 0000:0000  Imp  REGISTERPTRACE       (KERNEL.202)
 0000:0000  Imp  GETVERSION           (KERNEL.3)
 0000:0000  Imp  GETMODULEHANDLE      (KERNEL.47)
 0000:0000  Imp  __MOD_WINSOCK        (KERNEL.529)
 0000:0000  Imp  __MOD_DUSER          (KERNEL.523)
 0000:0000  Imp  __MOD_GDI            (KERNEL.524)
 0000:0000  Imp  __MOD_KERNEL         (KERNEL.520)
 0000:0000  Imp  __MOD_KEYBOARD       (KERNEL.526)
 0000:0000  Imp  __AHINCR             (KERNEL.114)
 0000:0000  Imp  WOW16CALL            (KERNEL.500)
 0000:0000  Imp  LOCALFREE            (KERNEL.7)
 0000:0000  Imp  GLOBALUNWIRE         (KERNEL.112)
 0000:0000  Imp  LSTRCMP              (USER.430)
 0000:0000  Imp  _WSPRINTF            (USER.420)
 0000:0000  Imp  __MOD_DGDI           (KERNEL.525)
 0000:0006  Abs  pLocalHeap
 0000:0008  Abs  pAtomTable
 0000:000A  Abs  pStackTop
 0000:000C  Abs  pStackMin
 0000:000E  Abs  pStackBot
 0000:9876  Abs  __acrtused2
 0000:9876  Abs  __ACRTUSED
 0000:9876  Abs  __fptaskdata
 0000:9876  Abs  __acrtmsg
 0000:D6D6  Abs  __aDBdoswp
 0001:0010       TOOLHELPLIBMAIN
 0001:016A       LIBENTRY
 0001:018A       WEP
 0001:01D6       KERNELTYPE
 0001:02A2       GLOBALINFO
 0001:0318       GLOBALFIRST
 0001:039A       GLOBALNEXT
 0001:0418       GLOBALENTRYHANDLE
 0001:04AA       GLOBALENTRYMODULE
 0001:0582       GLOBALHANDLETOSEL
 0001:0596       WALK386COUNT
 0001:05C1       WALK386FIRST
 0001:0615       WALK386
 0001:06D5       WALK386HANDLE
 0001:06FC       WALKLOC386COUNT
 0001:0723       WALKLOC386FIRST
 0001:074A       WALKLOC386
 0001:07F2       WALK386VERIFYLOCHEAP
 0001:084E       SELTOARENA386
 0001:08A2       NEXTLRU386
 0001:0914       LOCALINFO
 0001:0964       LOCALFIRST
 0001:09F0       LOCALNEXT
 0001:0A98       MODULEFIRST
 0001:0AE2       MODULENEXT
 0001:0B1E       MODULEFINDNAME
 0001:0B96       MODULEFINDHANDLE
 0001:0CBC       TASKFIRST
 0001:0D00       TASKNEXT
 0001:0D42       TASKFINDHANDLE
 0001:0D9A       TASKSETCSIP
 0001:0DCC       TASKGETCSIP
 0001:0DF8       TASKSWITCH
 0001:0E76       TS_FROMYIELD
 0001:0EA6       TASKINFO
 0001:0F5A       STACKTRACEFIRST
 0001:0FA6       STACKTRACECSIPFIRST
 0001:100A       STACKTRACENEXT
 0001:10EE       STACKFRAMEFIRST
 0001:117A       STACKFRAMENEXT
 0001:1210       SYSTEMHEAPINFO
 0001:12A2       USERGDIDGROUP
 0001:12CE       USERGDISPACE
 0001:1320       USERGDITYPE
 0001:13B2       MEMMANINFO
 0001:1468       HELPERVERIFYSEG
 0001:1482       HELPERHANDLETOSEL
 0001:14A6       HELPERVERIFYLOCHEAP
 0001:14B5       HELPERGLOBALTYPE
 0001:164E       HELPERGRABSELECTOR
 0001:1656       HELPERRELEASESELECTOR
 0001:1665       HELPERSETSIGNALPROC
 0001:1683       HELPERSIGNALPROC
 0001:1703       HELPERSEGLEN
 0001:1741       HELPERGETSEGNUMBER
 0001:177B       HELPERPDBTOTDB
 0001:17A8       WALK286COUNT
 0001:17D3       WALK286FIRST
 0001:181B       WALK286
 0001:18E4       WALK286HANDLE
 0001:1907       WALKLOC286COUNT
 0001:192E       WALKLOC286FIRST
 0001:1955       WALKLOC286
 0001:19F7       WALK286VERIFYLOCHEAP
 0001:1ABF       NEXTLRU286
 0001:1B30       NOTIFYREGISTER
 0001:1BE6       NOTIFYUNREGISTER
 0001:1C92       NOTIFYISHOOKED
 0001:1CB6       NOTIFYINIT
 0001:1D0D       NOTIFYUNINIT
 0001:1D4A       NOTIFYHANDLER
 0001:1E03       NOTIFYRIPHANDLER
 0001:1E5F       DECODENOTIFICATION
 0001:201A       INTERRUPTREGISTER
 0001:20CA       INTERRUPTUNREGISTER
 0001:2166       INTERRUPTISHOOKED
 0001:218A       INTERRUPTINIT
 0001:2218       INTERRUPTUNINIT
 0001:2260       GP_HANDLER
 0001:2260       INTERRUPTHANDLER
 0001:226A       GP_STDMODEHANDLER
 0001:2274       SF_HANDLER
 0001:227E       SF_STDMODEHANDLER
 0001:2288       PF_HANDLER
 0001:2292       PF_STDMODEHANDLER
 0001:229C       UD_HANDLER
 0001:22A6       INT1_HANDLER
 0001:22B0       INT3_HANDLER
 0001:22BA       CASRQ_HANDLER
 0001:22C4       DIV0_HANDLER
 0001:2349       COMMONINTERRUPTENTRY
 0001:23A0       DIH_NOTPVGPFAULT
 0001:23E2       DIH_NOTCASRQ
 0001:23EA       DIH_DPMICHAINON
 0001:23FF       DIH_FOUND
 0001:2413       DIH_EXCEPTION
 0001:242F       DIH_ENOUGHROOMONSTACK
 0001:2463       DIH_STACKOK
 0001:249C       DIH_BADSTACK
 0001:24F4       DIH_DPMIRESTART
 0001:2506       DIH_SKIPDPMI
 0001:252E       DIH_CALLBACKRESTART
 0001:255E       DIH_NEXTNOTFOUND
 0001:257E       DIH_NUKEIT
 0001:25A7       DIH_NUKEAPP
 0001:25B3       DIH_30STDCHAINON
 0001:25D9       DIH_CHAINON
 0001:25F4       DIH_NOCHAINADDR
 0001:25FD       DIH_EMULATEDPMI
 0001:2639       DIH_EMDPMIRESTART
 0001:2669       DIH_REBUILDDPMIFRAME
 0001:26AE       INTERRUPTINFO
 0001:26C8       TERMINATEAPP
 0001:2782       SIGNALREGISTER
 0001:2816       SIGNALUNREGISTER
 0001:288C       MEMORYREAD
 0001:2A34       MEMORYWRITE
 0001:2C30       MAKEALIAS
 0001:2C76       TIMERCOUNT
 0001:2D24       CLASSFIRST
 0001:2D31       CLASSNEXT
 0001:2D41       __wflags
 0001:2D44       __fstrncpy
 0001:2D6E       __NMSG_TEXT
 0001:2D99       __NMSG_WRITE
 0002:0004       rsrvptrs
 0002:0010       _szKernel
 0002:0038       WCASRQFLAG
 0002:003A       DWCASRQCSIP
 0002:003E       LPFNOLDPROC
 0002:005C       INTINFO
 0002:00AC       LPGDIFLAG
 0002:00B0       HGDI
 0002:00B6       LPFNPV
 0002:00BA       LPOLDHANDLER
 0002:00BE       LPCHAINCSIP
 0002:00D0       STKHQQ
 0002:00D2       __adbgmsg
 0002:00D4       ___aDBswpflg
 0002:00D6       ___aDBswpchk
 0002:00D8       __aDBrterr
 0002:00DA       ___aDBexit
 0002:00E8       __caption
 0002:0180       __edata
 0002:0180       _wLibInstalled
 0002:0180       _edata
 0002:0182       _lpfnUserSeeUserDo
 0002:0186       _lpfntimeGetTime
 0002:018A       _NPNOTIFYNEXT
 0002:018C       _hGDIHeap
 0002:018E       _npwTDBHead
 0002:0190       _npdwSelTableStart
 0002:0192       _lpfnNotifyHook
 0002:0196       _hMaster
 0002:0198       _npwTDBCur
 0002:019A       _lpfnGetFreeSystemResources
 0002:019E       _wSel
 0002:01A0       _NPSIGNALHEAD
 0002:01A2       _lpfnFatalExitHook
 0002:01A6       _WINTINSTALLED
 0002:01A8       _NPNOTIFYHEAD
 0002:01AA       _lpfnGetUserLocalObjType
 0002:01AE       _hUserHeap
 0002:01B0       _wTHFlags
 0002:01B2       _wLRUCount
 0002:01B4       _NPINTHEAD
 0002:01B6       _WNOTIFYINSTALLED
 0002:01B8       _npwSelTableLen
 0002:01BA       _WSIGNALINSTALLED
 0002:01BC       _npwExeHead
 0002:01BE       _segKernel
 0002:01C0       __end
 0002:01C0       _end

Program entry point at 0001:016a
